:020000040000FA
:0414000007EF0AF0F8
:0A14080053821BED34F0ECEF32F0DC
:10141600000100B314A5147914501405010905A19F
:101426000105091901290615002501350045017533
:101436000195068102950281010600FF090115004A
:1014460026FF00750895019100C0090229000101D7
:101456000080320904000002030000000921110186
:101466000001222F00070581034000010705010343
:101476004000011A0342004900410020004D006966
:1014860000630072006F0044004400520012010025
:101496000200000008D804EEEC0100010200010E73
:1014A6000348006F006E006D0061006E00040309C2
:0214B600040030
:1065A2008150FF0A3F0B1200C150F00B0709C16E68
:1065B2003F0E9312F19E1200010E3626000E372274
:1065C200382239224950D8A41200402A4050D8A477
:1065D20012004068120000EE60F01E0EEE6AE8063D
:1065E200FDE100EE36F01D0EEE6AE806FDE1539085
:1065F2005392000EF86E0001F7EF33F06984689849
:106602006D82010E496E000E406E000E0E6E750E0A
:106612000D6E000E0F6E000E106E000E126E000E4A
:10662200116E76EC34F012004D50D8A41200000E18
:106632006D6E000E696E160E6F6E9F0E6B6E7B0E88
:10664200696ED08EA28AA08AF28E01D06D866DA666
:10665200FDD7010E4D6E1200000E496E000E0E6E39
:10666200740E0D6E000E0F6E000E106E000E126E86
:10667200000E116E76EC34F06D92699401D068943C
:1066820068B4FDD7000E406E1200000E0001786F54
:10669200000E796F1E0E096E010E7AEC33F0000EB9
:1066A200016E000E026E050E036E010E046E010EE7
:1066B200B7EC39F001C076F002C077F01200000E9C
:1066C2000001786F000E796F1E0E7E6F010E96EC40
:1066D20033F0000E2A6E000E2B6E050E2C6E010E8C
:1066E2002D6E010E38EC3AF02AC076F02BC077F00E
:1066F20012000C6E09A405D0000E016E0C50ECECD9
:1067020034F009A205D0010E016E0C50ECEC34F00D
:10671200700E0C240A6E0B6A0F0E0B220AC0D9FFF0
:106722000BC0DAFF09C0DFFF1200346E00017EA544
:1067320005D0000E2A6E345036EC35F000017EA3EF
:1067420005D0010E2A6E345036EC35F0700E34242A
:10675200326E336A0F0E332232C0D9FF33C0DAFFF2
:106762007EC0DFFF120070A01DD03EC0D9FF3FC027
:10677200DAFF800EDE18D8A414D06EC0D9FF6FC025
:10678200DAFF840EDE18D8A40CD03EC0D9FF3FC079
:10679200DAFF0C0EDF6E3EC0D9FF3FC0DAFF000EFB
:1067A200DB8E7090689A120003C009F004C00AF0F0
:1067B20001C007F002C008F010D009C0D9FF0AC01A
:1067C200DAFFDF500B6E094A0A2A07C0D9FF08C058
:1067D200DAFF0BC0DFFF074A082A0506D8A0060623
:1067E2000528EBE10628D8B41200E7D7D5EC32F041
:1067F20060EC33F0D0EC3BF015EC33F01F0E4D643F
:1068020001D002D0010E01D0000E0001806F816B19
:106812006DA203D0826B822B02D00001826B825167
:106822008013000E811380518111D8A4E7D7CBECDD
:1068320035F0E4D70600E1CF20F0E2CF21F0D9CF46
:1068420022F0DACF23F0F3CF24F0F4CF25F0F6CF05
:1068520026F0F7CF27F0F8CF28F0F5CF29F03EEC5D
:106862003BF029C0F5FF28C0F8FF27C0F7FF26C07C
:10687200F6FF25C0F4FF24C0F3FF23C0DAFF22C0D5
:10688200D9FF21C0E2FF20C0E1FF53921100020EA6
:106892004B18D8A403D0B9EC3AF01200000E4B6E9C
:1068A2004750D8A41FD020EE01F03C50D9263D50CD
:1068B200DA22080EDF6E20EE02F03C50D9263D505F
:1068C200DA22200EDE6E040EDD6E3CC0D9FF3DC022
:1068D200DAFF0C0EDF6E3CC0D9FF3DC0DAFF000EBE
:1068E200DB8E1200000E476E120006D046EC33F02B
:1068F20012003AEC39F012000DC013F00EC014F081
:106902001450000AD8B404D07F0AD8A4120018D0B8
:106912001350010AD8B4EAD7030AD8B41200010A04
:10692200D8B4E7D7060AD8B41200770AD8B412004E
:10693200010AD8B41200070AD8B41200010A1200E0
:106942001350FF0A1200000E4C6E000E456E000E30
:10695200426E000E416E000E476E000E4B6E6EC010
:10696200D9FF6FC0DAFF7F0EDF16040E00016E1929
:106972006E6F6F516F6F6EC0D9FF6FC0DAFF7F0EFF
:10698200DF16040E6E196E6F6F516F6F3CC0D9FF28
:106992003DC0DAFF7F0EDF16000E6B6F000E6D6FCB
:1069A200000E6C6F000E636F000E656F000E646F59
:1069B200C8EC38F0000E0E6E030E0D6E000E0F6E58
:1069C200000E106E000E126E000E116E76EC34F098
:1069D20058EC38F01200066E000E076E040E086EB8
:1069E2000150026E036AD890023603360650046ED6
:1069F200056AD89004360536D8900436053602501A
:106A0200042603500522D89004360536D890043661
:106A12000536045007260550082207C0D9FF08C0D2
:106A2200DAFFDF9E0150D8A407D00650020D720E85
:106A3200F324D96E000E06D00650020D6E0EF3241A
:106A4200D96E000EF420DA6E07C0DEFF08C0DDFF4B
:106A520007C0D9FF08C0DAFFDF9C20EE04F0075020
:106A6200D9260850DA22DF8C12002F6E000E306E0B
:106A7200040E316E2A502B6E2C6AD8902B362C368F
:106A82002F502D6E2E6AD8902D362E36D8902D3658
:106A92002E362B502D262C502E22D8902D362E36C7
:106AA200D8902D362E362D5030262E50312230C021
:106AB200D9FF31C0DAFFDF9E2A50D8A407D02F5069
:106AC200020D720EF324D96E000E06D02F50020D65
:106AD2006E0EF324D96E000EF420DA6E30C0DEFFA3
:106AE20031C0DDFF30C0D9FF31C0DAFFDF9C20EEBC
:106AF20004F03050D9263150DA22DF8C12002D0EEC
:106B0200466E50C01EF0FD0E1E16D8A43BD050C0DB
:106B12001EF0D8901E323F0E1E161E50040D000E9F
:106B2200F3243E6E040EF4203F6E3EC03CF03FC0A4
:106B32003DF0040E3C183C6E3D503D6E3EC0D9FF08
:106B42003FC0DAFFDF30E8320F0B0D0AD8A417D0AE
:106B5200200E016E040E026E20EE02F03E50D92687
:106B62003F50DA22DECF03F0DDCF04F0000E066ED6
:106B7200080E056ED5EC33F0A4EC34F0120048ECAC
:106B820034F012005050FD0B040AD8A41200C5ECD8
:106B920036F01200000176517711D8B40AD076C0CF
:106BA200D9FF77C0DAFFDFAE04D01FD018EF00F0B4
:106BB2000DD00501005100017E6F7F6B7F51000AED
:106BC200D8A404D07E51BB0AD8B4F0D7000E2A6EE6
:106BD200000E2B6E050E2C6E010E2D6E010E38EC82
:106BE2003AF02AC076F02BC077F000017851791183
:106BF200D8B406D078C0D9FF79C0DAFFDFBE120060
:106C0200D1EC32F0356E35C040F5010E2A6E400EE1
:106C12002B6E050E2C6E010E2D6E010E38EC3AF025
:106C22002AC078F02BC079F01200000E426E000EDE
:106C3200416E020E4B18D8A41FD020EE01F03C503A
:106C4200D9263D50DA22080EDF6E20EE02F03C50CB
:106C5200D9263D50DA22280EDE6E040EDD6E3CC0CF
:106C6200D9FF3DC0DAFF480EDF6E3CC0D9FF3DC000
:106C7200DAFF000EDB8E120000016C510401265D6A
:106C820000016D5104012759D8B004D026C46CF01C
:106C920027C46DF088EC37F0000120EE02F06E514F
:106CA200D9266F51DA22280EDE6E040EDD6E6EC01A
:106CB200D9FF6FC0DAFF480EDF6E6EC0D9FF6FC01A
:106CC200DAFF000EDB8E1200000E0401286F000EA8
:106CD200296F3DD000016B8F4A04D8A44AD0040129
:106CE200288347D000016B8F44D000016B8F0401D1
:106CF20024510F0B0009D8B43CD024BF0AD0245130
:106D02000F0B016E0150020D720EF324D96E000EAC
:106D120009D024510F0B016E0150020D6E0EF324A7
:106D2200D96E000EF420DA6EDECF03F0DDCF04F070
:106D320003C0D9FF04C0DAFFDFAE1BD003C0D9FF06
:106D420004C0DAFFDFA415D0010E286F12D0205143
:106D52001F0B016E026A0250000AD8A40AD0015029
:106D6200000AD8B4B7D7010AD8B4BCD7030AD8B43A
:106D7200BCD700016BAF1200280E686F040E696F5A
:106D82006B81020E6C6F12006EC0D9FF6FC0DAFF0A
:106D92000001000EDFBC010E026E040E6E196E6F52
:106DA2006F516F6F080E4D18D8A40BD004012251F9
:106DB2007F0B6E6E6E50D8B402D0100E01D0040E4E
:106DC2004D6E4B04D8A43BD0000120EE02F06E5170
:106DD200D9266F51DA22280EDE6E040EDD6E88ECA3
:106DE20037F0020E4C18D8A40DD06EC0D9FF6FC078
:106DF200DAFF040EDF6E6EC0D9FF6FC0DAFF000E3D
:106E0200DB8E12000250D8A40DD06EC0D9FF6FC025
:106E1200DAFF480EDF6E6EC0D9FF6FC0DAFF000ED8
:106E2200DB8E12006EC0D9FF6FC0DAFF080EDF6E74
:106E32006EC0D9FF6FC0DAFF000EDB8E12000001B8
:106E420063BF639F000E4B6E12004450D8A4120021
:106E5200010E446E4350D8A41200010E436E020E7E
:106E62004B18D8A416D0000120EE01F06E51D9269D
:106E72006F51DA22000EDF6E6EC0D9FF6FC0DAFFEB
:106E8200480EDF6E6EC0D9FF6FC0DAFF000EDB8ED8
:106E920012004B04D8A41200000E476E20EE01F03F
:106EA2003E50D9263F50DA22080EDF6E20EE02F065
:106EB2003E50D9263F50DA22200EDE6E040EDD6EE1
:106EC2003EC0D9FF3FC0DAFF040EDF6E3EC0D9FFDD
:106ED2003FC0DAFF000EDB8E010E476E20EE01F09E
:106EE2003C50D9263D50DA22080EDF6E20EE02F029
:106EF2003C50D9263D50DA22200EDE6E040EDD6EA5
:106F02003CC0D9FF3DC0DAFF800EDF6E1200080ED2
:106F1200016E00016D5110E1080E6C5DD8B00CD00D
:106F22006CC001F04C50D8A402D0010E04D04C0425
:106F3200D8A402D0020E4C6E01506C5F000E6D5B45
:106F420020EE01F06E51D9266F51DA2201C0DFFF27
:106F5200280E3A6E040E3B6E6BA11CD03AD068C06C
:106F6200F6FF69C0F7FFF86A3AC0D9FF3BC0DAFF03
:106F7200070EF76403D00800F55005D0F6CFE1FF05
:106F8200F7CFE2FFE750DF6E0001684B692B3A4A08
:106F92003B2A01060150D8B41200E1D768C0F6FFBF
:106FA20069C0F7FFF86A3AC0D9FF3BC0DAFF070EA3
:106FB200F76403D00800F55005D0F6CFE1FFF7CF14
:106FC200E2FFE750DF6E0001684B692B3A4A3B2A29
:106FD20001060150D8B41200E1D700016B8F710E87
:106FE200016E0F0E026E000E046E000E036E000E96
:106FF200066E010E056EFBEC3CF0000E016E040EF7
:10700200026E000E046E000E036E000E066E200E5F
:10701200056EFBEC3CF06D8C000E156E7C0E15249B
:10702200D96EDA6A000EDA22000EDF6E7A0E1524AD
:10703200D96EDA6A000EDA22000EDF6E152A010E10
:107042001564ECD7510E016E000E026E000E046E36
:10705200000E036E000E066E010E056EFBEC3CF098
:107062006D9C080E00016E6F040E6F6F000E3E6E77
:10707200040E3F6E3EC03CF03FC03DF022C452F0D1
:107082005250D8A403D0100E4D6E1200000E0E6E98
:10709200010E0D6E520E0F6E000E106E000E126E6D
:1070A200010E116E76EC34F0200E4D6E12006D98CA
:1070B20000016BBF38D063AF0BD0020E4B6E415054
:1070C200D8B416EC36F0000E436E000E446E120079
:1070D20020EE01F03C50D9263D50DA22080EDF6E38
:1070E20020EE02F03C50D9263D50DA22200EDE6E10
:1070F200040EDD6E3CC0D9FF3DC0DAFF0C0EDF6E20
:107102003CC0D9FF3DC0DAFF000EDB8E6EC0D9FF56
:107112006FC0DAFF040EDF6E6EC0D9FF6FC0DAFFF8
:10712200000EDB8E1200040120AF10D0010E4B6E58
:107132004250D8B416EC36F0000E436E000E446E88
:107142004550D8A4120026EC37F01200020E4B6E06
:1071520020EE01F03C50D9263D50DA22080EDF6EB7
:1071620020EE02F03C50D9263D50DA22200EDE6E8F
:10717200040EDD6E3CC0D9FF3DC0DAFF040EDF6EA7
:107182003CC0D9FF3DC0DAFF000EDB8ED5D704012B
:107192002039E832030B0009D8A4120042D00001C2
:1071A2006B8F080E4D6E12002DEC3EF01200EEECCD
:1071B20037F01200520E0001686F000E696F6B818A
:1071C200010E6C6F6B8F120065EC36F01200C9EC89
:1071D2003EF01200510E24250001686F696B000E0B
:1071E20069236B81010E6C6F6B8F120000016B8F34
:1071F200510E04012425D96EDA6A000EDA2222C465
:10720200DFFF1200000E0E6E020E0D6E000E0F6EEC
:10721200000E106E000E126E000E116E76EC34F03F
:10722200120021511C6E1D6A1D50000AD8A41200C2
:107232001C50000AD8B4C8D7010AD8B4C8D7020A69
:10724200D8B4C5D7060AD8B4AAD7030AD8B4ACD7DB
:10725200010AD8B4D7D70F0AD8B4ACD7010AD8B428
:10726200A6D7030AD8B4B6D7010AD8B4BFD7070A3B
:107272001200040120511F0BE806D8A41200245169
:10728200D8A41200060E2119D8B41AD028D052045C
:10729200D8A425D0620E0001686F140E696F000E2B
:1072A2006D6F090E0BD0C00E6B6F19D0210E00014D
:1072B200686F140E696F000E6D6F2F0E6C6FF3D72F
:1072C2002351016E026A0250000AD8A408D001506C
:1072D200210AD8B4DCD7030AD8B4E8D7010A0401DA
:1072E2002039E832030BE806D8A4120024D04F0E4E
:1072F2000001686F000E696F000E6D6F010E6C6FFA
:10730200C10E6B6F1200800E00016B6F23C44FF031
:1073120012004E0E0001686F000E696F000E6D6F55
:10732200010E6C6F810E6B6F1200800E00016B6F8D
:1073320022C44EF012002151016E026A0250000A6C
:10734200D8A412000150010AD8B41200030AD8B41A
:10735200CED7010AD8B4DDD70A0AD8B41200030A7C
:10736200D8B4D1D7010AD8A41200DFD7096E0150D0
:10737200D8B407D00950020D6E0EF324D96E000E58
:1073820006D00950020D720EF324D96E000EF420BD
:10739200DA6EDECF0AF0DDCF0BF00A500B10D8A464
:1073A20005D0000E016E000E026E120020EE02F0F9
:1073B2000A50D9260B50DA2202C0DEFF03C0DDFFDD
:1073C20020EE01F00A50D9260B50DA2204C0DFFF6A
:1073D2000AC0D9FF0BC0DAFF400EDF160AC0D9FF80
:1073E2000BC0DAFF000EDB860AC0D9FF0BC0DAFF42
:1073F200000EDB8E0150D8B418D00950020D6E0E6B
:10740200F324D96E000EF420DA6EDECF05F0DDCF64
:1074120006F0040E0518076E0650086E0950020D9C
:107422006E0EF324D96E000E17D00950020D720EA3
:10743200F324D96E000EF420DA6EDECF05F0DDCF34
:1074420006F0040E0518076E0650086E0950020D6C
:10745200720EF324D96E000EF420DA6E07C0DEFF3E
:1074620008C0DDFF0AC001F00BC002F01200326E4C
:107472002A50D8B407D03250020D6E0EF324D96EC2
:10748200000E06D03250020D720EF324D96E000E99
:10749200F420DA6EDECF33F0DDCF34F03350341027
:1074A200D8A405D0000E2A6E000E2B6E120020EE1C
:1074B20002F03350D9263450DA222BC0DEFF2CC022
:1074C200DDFF20EE01F03350D9263450DA222DC0F0
:1074D200DFFF33C0D9FF34C0DAFF400EDF1633C0FE
:1074E200D9FF34C0DAFF000EDB8633C0D9FF34C0C7
:1074F200DAFF000EDB8E2A50D8B418D03250020DBB
:107502006E0EF324D96E000EF420DA6EDECF2EF06A
:10751200DDCF2FF0040E2E18306E2F50316E325008
:10752200020D6E0EF324D96E000E17D03250020DEA
:10753200720EF324D96E000EF420DA6EDECF2EF036
:10754200DDCF2FF0040E2E18306E2F50316E3250D8
:10755200020D720EF324D96E000EF420DA6E30C0E2
:10756200DEFF31C0DDFF33C02AF034C02BF0120041
:1075720020EE01F03E50D9263F50DA22DF50026E53
:1075820002500001645D000E6559D8A064C002F08B
:107592000250645F000E655B000E016E0FD0280E74
:1075A2000124D96EDA6A040EDA2260C0E1FF61C0FA
:1075B200E2FFDFCFE7FF604B612B012A0250015C43
:1075C200D8A0EDD764516511D8B432D020EE01F0C5
:1075D2003C50D9263D50DA22080EDF6E20EE02F032
:1075E2003C50D9263D50DA22280EDE6E040EDD6EA6
:1075F2003EC0D9FF3FC0DAFFDFBC0DD03CC0D9FF8F
:107602003DC0DAFF480EDF6E3CC0D9FF3DC0DAFF55
:10761200000EDB8E12003CC0D9FF3DC0DAFF080E1F
:10762200DF6E3CC0D9FF3DC0DAFF000EDB8E1200D8
:1076320020EE01F03C50D9263D50DA22080EDF6ED2
:1076420020EE02F03C50D9263D50DA22200EDE6EAA
:10765200040EDD6E3CC0D9FF3DC0DAFF040EDF6EC2
:107662003CC0D9FF3DC0DAFF000EDB8E639F455060
:10767200D8A4120026EC37F012004D04D8B46DBA2B
:1076820006D0000E686E69806988020E4D6E68B47D
:1076920069A403D068942DEC33F06DA202D0A19AB4
:1076A200120068B069A006D065EC3CF0A08A040E16
:1076B2004D6E689068B869A802D0FFEC32F068ACF1
:1076C2001AD069AC0ED0000E0E6E730E0D6E000E47
:1076D2000F6E000E106E000E126E010E116E76EC21
:1076E20034F0689CDDEC32F04650D8A44606465091
:1076F200D8B426EC37F068BA69AA02D0B4EC33F0F9
:1077020068B269A20FD07F0E0E6E0D68000E0F6E6A
:10771200000E106E000E126E010E116E76EC34F039
:10772200000E6A6E040E4D6002D0A19A120069A684
:1077320034D0000E1F6E68A630D06CCF50F050309F
:10774200E832E8320F0B486E689650B406D07A0ED3
:107752004824D96EDA6A000E05D07C0E4824D96E10
:10776200DA6A000EDA220001DF704850D8A403D092
:1077720080EC35F00ED0000E0E6E720E0D6E500EB5
:107782000F6E000E106E000E126E000E116E76EC71
:1077920034F01F2A030E1F64CED7A19A1200A09ABA
:1077A200000E6A6E000E686E000E706E710E2A6E0A
:1077B2000F0E2B6E000E2D6E000E2C6E000E2F6E15
:1077C200010E2E6E94EC3DF0160E6F6E9F0E6B6ED8
:1077D2007B0E696E000E00017E6F7E51040D000E5D
:1077E200F324D96E040EF420DA6EDE6ADE6ADE6AF3
:1077F200DD6A7E2B070E7E65F0D76D8C000E6E6EF5
:107802006D986D9C6896000E6B6F000E636F000E94
:10781200656F000E646F68B6F5D7010E446E010EF7
:10782200436E000E426E000E416E000E496E000E57
:107832007E6F7E51020D6E0EF324D96E000EF4207F
:10784200DA6E000EDE6E000EDD6E7E51020D720EDD
:10785200F324D96E000EF420DA6E000EDE6E000EF6
:10786200DD6E7C0E7E25D96EDA6A000EDA22000EFB
:10787200DF6E7A0E7E25D96EDA6A000EDA22000EEB
:10788200DF6E7E2B010E7E65D4D7080E6E6F040E5E
:107892006F6F160E706E040E0401036F200E026FDE
:1078A200080E016F040E006F008F000E526E000E64
:1078B200366E000E376E000E386E000E396E000EF8
:1078C200406E000E4D6E1200A09A000E6A6E000EFF
:1078D200686E000E706E710E016E0F0E026E000E5B
:1078E200046E000E036E000E066E010E056EFBECBA
:1078F2003CF0160E6F6E9F0E6B6E7B0E696E000E65
:107902000D6E0D50040D000EF324D96E040EF420FA
:10791200DA6EDE6ADE6ADE6ADD6A0D2A070E0D6441
:10792200F0D76D8C000E6E6E6D986D9C6896000E91
:1079320000016B6F000E636F000E656F000E646FC7
:1079420068B6F4D7010E446E010E436E000E426E0D
:10795200000E416E000E496E000E0D6E0D50020DAE
:107962006E0EF324D96E000EF420DA6E000EDE6E77
:10797200000EDD6E0D50020D720EF324D96E000E54
:10798200F420DA6E000EDE6E000EDD6E7C0E0D242B
:10799200D96EDA6A000EDA22000EDF6E7A0E0D243C
:1079A200D96EDA6A000EDA22000EDF6E0D2A010E9F
:1079B2000D64D4D7080E00016E6F040E6F6F160EA1
:1079C200706E040E0401036F200E026F080E016F29
:1079D200040E006F008F000E526E000E366E000E07
:1079E200376E000E386E000E396E000E406E000EBD
:1079F2004D6E120001C00BF002C00CF005500610D3
:107A0200D8B412000BC0D9FF0CC0DAFF03C0DFFFED
:107A120005500B24076E06500C20086EFF0E07243B
:107A2200D96EFF0E0820DA6E03C0DFFF065004E1B4
:107A3200030E055CD8A0120020EE01F00B50D926EF
:107A42000C50DA2203C0DFFF20EE02F00B50D926E1
:107A52000C50DA2203C0DFFF05500B24076E0650DC
:107A62000C20086EFE0E0724D96EFF0E0820DA6E77
:107A720003C0DFFF05500B24076E06500C20086E72
:107A8200FD0E0724D96EFF0E0820DA6E03C0DFFF59
:107A9200065004E1070E055CD8A0120020EE03F0A8
:107AA2000B50D9260C50DA2203C0DFFF05500B24FD
:107AB200076E06500C20086EFC0E0724D96EFF0ECE
:107AC2000820DA6E03C0DFFF065004E1090E055CF0
:107AD200D8A012000BC007F00CC008F0071E081E49
:107AE200074A082A030E0714096E0A6A09500B2670
:107AF2000A500C220950055E0A50065AFC0E051661
:107B0200FF0E06160BD00BC0D9FF0CC0DAFF03C064
:107B1200DFFF0506D8A006060B4A0C2A0550061000
:107B2200D8B41200F0D72AC034F02BC035F02E5052
:107B32002F10D8B4120034C0D9FF35C0DAFF2CC0E0
:107B4200DFFF2E503424306E2F503520316EFF0E61
:107B52003024D96EFF0E3120DA6E2CC0DFFF2F5099
:107B620004E1030E2E5CD8A0120020EE01F0345086
:107B7200D9263550DA222CC0DFFF20EE02F0345035
:107B8200D9263550DA222CC0DFFF2E503424306E35
:107B92002F503520316EFE0E3024D96EFF0E31206B
:107BA200DA6E2CC0DFFF2E503424306E2F50352079
:107BB200316EFD0E3024D96EFF0E3120DA6E2CC0EC
:107BC200DFFF2F5004E1070E2E5CD8A0120020EE3A
:107BD20003F03450D9263550DA222CC0DFFF2E5064
:107BE2003424306E2F503520316EFC0E3024D96E85
:107BF200FF0E3120DA6E2CC0DFFF2F5004E1090E98
:107C02002E5CD8A0120034C030F035C031F0301EE6
:107C1200311E304A312A030E3014326E336A32502A
:107C220034263350352232502E5E33502F5AFC0EFA
:107C32002E16FF0E2F160BD034C0D9FF35C0DAFF37
:107C42002CC0DFFF2E06D8A02F06344A352A2E502C
:107C52002F10D8B41200F0D7800E04012019D8A436
:107C62001200C00E00016B6F80D0930E0001686F8E
:107C7200140E696F000E6D6F120E6C6F120022519E
:107C8200D8A440D02251020D1F0EF324F66E140E1A
:107C9200F420F76E0900F5CF68F00A00F5CF69F01D
:107CA200020E00016825016E000E6921026E01C0FC
:107CB200F6FF02C0F7FFF86A070EF76403D0080068
:107CC200F55005D0F6CFE1FFF7CFE2FFE750000114
:107CD2006C6F030E6825016E000E6921026E01C0F1
:107CE200F6FF02C0F7FFF86A070EF76403D0080038
:107CF200F55005D0F6CFE1FFF7CFE2FFE7500001E4
:107D02006D6F1200000E00016B6F1200030E2261F4
:107D120024D02251020D190EF324F66E140EF42013
:107D2200F76E0900F5CF68F00A00F5CF69F068C078
:107D3200F6FF69C0F7FFF86A070EF76403D0080080
:107D4200F55005D0F6CFE1FFF7CFE2FFE750016E25
:107D5200015000016C6F6D6B1200000E00016B6F21
:107D62001200000E00016B6F120004012351016E1C
:107D7200026A0250000AD8A4F4D70150010AD8B40A
:107D820074D7030AD8B47BD7010AD8B4BFD7E9D7CE
:107D920004012205D8A410D020511F0B0009D8A439
:107DA2000BD000016B8F030E04012119D8A402D05D
:107DB200010E01D0000E4A6E2251D8A412002051A9
:107DC2001F0B020AD8A4120024510F0B0009D8B4C9
:107DD200120024510F0B156E020E15601200200EB8
:107DE2004D18D8A4120000016B8F040124BF18D0D3
:107DF20024510F0B156E1550020D720EF324D96E1D
:107E0200000EF420DA6EDECF1AF0DDCF1BF0245123
:107E12000F0B156E166A7A0E1524D96E000E17D046
:107E220024510F0B156E1550020D6E0EF324D96EF0
:107E3200000EF420DA6EDECF1AF0DDCF1BF02451F3
:107E42000F0B156E166A7C0E1524D96E000E1620C5
:107E5200DA6EDF50196E19B006D0FB0E1A141A6EC4
:107E6200FF0E1B1404D0040E1A101A6E1B501B6E48
:107E720024BF0AD024510F0B156E1550020D720E3D
:107E8200F324D96E000E09D024510F0B156E155034
:107E9200020D6E0EF324D96E000EF420DA6E1AC0B3
:107EA200DEFF1BC0DDFF030E2119D8A42AD01AC0A1
:107EB200D9FF1BC0DAFFDFAE17D024BF09D024518F
:107EC2000F0B156E166A7A0E1524D96E000E08D0A5
:107ED20024510F0B156E166A7C0E1524D96E000EF6
:107EE2001620DA6E0001DF821AC0D9FF1BC0DAFF4A
:107EF200000EDB841AC0D9FF1BC0DAFF000EDB8E36
:107F02001200040E1A181A6E1B501B6E1AC0D9FFEB
:107F12001BC0DAFFDFAE1BD01AC0D9FF1BC0DAFFCD
:107F22007F0EDF161AC0D9FF1BC0DAFF000EDB8CF2
:107F3200000E0E6E050E0D6E1AC00FF01BC010F073
:107F4200000E126E020E116E76EC34F006D01AC0DC
:107F5200D9FF1BC0DAFF000EDB8C040E1A181A6E52
:107F62001B501B6E19B206D01AC0D9FF1BC0DAFF14
:107F7200DFAE2DD0040124BF09D024510F0B156EA2
:107F8200166A7A0E1524D96E000E08D024510F0BF2
:107F9200156E166A7C0E1524D96E000E1620DA6E46
:107FA2000001DF921AC0D9FF1BC0DAFF3B0EDF16B9
:107FB200000E0E6E050E0D6E1AC00FF01BC010F0F3
:107FC200000E126E020E116E76EC34F006D01AC05C
:107FD200D9FF1BC0DAFF3B0EDF16040124510F0B41
:107FE200156E166A700E1524176E0F0E1620186E77
:0E7FF20017C0D9FF18C0DAFFFE0EDF1612000E
:020000040020DA
:08000000FFFFFFFFFFFFFFFF00
:020000040030CA
:0E0000002A0C3F1EFF8381FF0FC00FE00F4050
:00000001FF
